:020000040000FA
:06000000542841302B30B2
:08000800A000030EA100831209
:100010000C1C2328DD1B23288E015C1C15285C107A
:100020005A088F005D0985051B285C145B088F004A
:100030005D088504DC170C108B180828210E83003E
:10004000A00E200E09008B1C49288B1031182E2879
:10005000B11C492864300102031C48282F2830288D
:100060003128322833283428352836283110B11465
:10007000A810031005190314AA0DA90DA80DB00BA3
:10008000492831152A08AF002908AE002808AD001C
:10009000B11081010B11210E8300A00E200E09006A
:0800A800203084008001840A6D
:1000B00060300402031C56281230B00074228316EC
:1000C000FF239000831283160C308505870183126D
:1000D00085018701073099000030831691009F0049
:1000E0008312C830831681008312013090000130E2
:1000F00083168C00831210308B00BD1B8128851D58
:1001000008233D1BBE013D1BBF013D1F0023810194
:100110008E018F010B118B100B108C130C138C1193
:100120000C100B178B17A5203119BB204822B30BDD
:10013000A128031085190314BA0DF0303A020319EF
:10014000A821DC183A2348239328640031180800BA
:100150000B1D08000B11B11031141230B000051D39
:10016000B628321483160113831208003210831646
:10017000011783120800321CC2282D090339AD0073
:10018000AE09AF09E4302F02F0300319AF004C3054
:100190002F020C300319AF006C302F023C300319D2
:1001A000AF00EC302F02FC300319AF00B3302F0248
:1001B000F3300319AF001B302F020F300319AF00CB
:1001C0003B302F023F300319AF00BB302F02FF300E
:1001D0000319AF0031110130B7008B1320303707FE
:1001E00083169B001C141A088312A400A500251076
:1001F0001030370783169B001C141A088312A300C3
:100200000030370783169B001C141A088312A200C3
:100210008B1722082D02031DA22923082E06FC3964
:10022000031DA229013003303702031D3B29003092
:100230002E060339031D2029BF1F2929BF13B1171B
:1002400003302E060339031D2929BF1B2929BF1797
:10025000B11744302F065439031D32293F1F0800BF
:100260003F13B11710302F065439031D3B293F1B94
:1002700008003F17B117AF13AF12AF11AF1024082A
:100280002F02031D702901303702031D4C293E182F
:100290004C293E14B1178E2202303702031D552916
:1002A000BE185529BE14B117A22203303702031D10
:1002B0005E293E195E293E15B117B6220430370279
:1002C000031D6729BE196729BE15B117CA2205305B
:1002D0003702031D70293E1A70293E16B117DE221F
:1002E00025082F02031DA22901303702031D7D2995
:1002F0003E1C7D293E10B117E82202303702031D53
:100300008629BE1C8629BE10B117EB2203303702A6
:10031000031D8F293E1D8F293E11B117EE22043097
:100320003702031D9829BE1D9829BE11B117F2226C
:1003300005303702031DA1293E1EA1293E12B11727
:10034000F622A229B70A0630370203180800ED2862
:100350000B13DD17B601B3019630B4000130B500C0
:100360000130B70085018701B1131D22A520B30B11
:10037000D329031085190314BA0DF0303A0203197A
:100380000B2AB41F8501B41F8701B40BD32937088A
:10039000B6080319B6000319D129FF30850087007C
:1003A000B6039630B400311DB6293111321CDD2957
:1003B0002D090339AD00AE09AF0951302F0655396B
:1003C0000319F22905302F0655390319F229153082
:1003D0002F0655390319F22955302F0655390319BF
:1003E000F229B629AF13AF12AF11AF108B13203023
:1003F0003707BC002F08BB00562210303707BC005F
:100400002E08BB00562200303707BC002D08BB0069
:1004100056228B17172285018701B70AB6010630CD
:100420003702031CB6290B17DD1300230800053023
:10043000370203190800850187016430B9003330A1
:100440008F1F85008F1B8501A520311D1F2A3111AB
:10045000321C2F2A2D090339AD00AE09AF095130E6
:100460002F06553903191D2A05302F065539031952
:100470001D2A15302F06553903191D2A55302F0610
:10048000553903191D2AB90B1F2A85018701080058
:10049000B11F0800B1131030BC003E08BB0056224B
:1004A0003030BC003F08BB00562208003C088B13CC
:1004B00083169B001C141A0883128B173B02031926
:1004C00008008B133B0883161C159A003C089B0000
:1004D00055309D00AA309D009C1464009C186D2A24
:1004E0001C1183128B1708000A30DE007D30DF00FC
:1004F000831600309B001C141A088312BD0083165B
:1005000010309B001C141A088312BE008316303072
:100510009B001C141A088312BF0008000730C1009A
:10052000D2100E303E05031D08008B1383162030B9
:100530009B001C141A088312D6008B178E018F01A2
:100540000C1008000630C20052110D303E05031D8C
:1005500008008B13831620309B001C141A0883128A
:10056000D6008B178E018F010C1008000730C300D6
:10057000D2110B303E05031D08008B13831620306B
:100580009B001C141A088312D6008B178E018F0152
:100590000C1008000530C400521207303E05031D40
:1005A00008008B13831620309B001C141A0883123A
:1005B000D6008B178E018F010C1008008B13831649
:1005C00040309B001C141A088312D1008B170800BE
:1005D0008512DD12080005125D120800DC1C851072
:1005E000DD100800DC1C05105D1008008B1383165D
:1005F00041309B001C141A088312D1008B1708008D
:10060000C101C201C301C4013E1EF62ADE2A080050
:10061000B601B301B4013D1C102B3D10BD141D2BC0
:10062000BD1C152BBD103D151D2B3D1D1A2B3D115D
:10063000BD151D2BC030BD053D143D083F39B6002A
:100640006400222B232B242B252B262B3330B41B89
:100650008500B41F8501B30B202BB40B202B031096
:10066000B60CB608031D202B0030BC003D08BB00B3
:1006700056220800BF1F452B3F1B85103F1B05144A
:100680003F1F85143F1F0510080085100510080046
:10069000DC10BD18DC14BD19DC145108FF3CDB0074
:1006A000F0305107DA000F303E0503190800D60874
:1006B0000319632BDC1F0800DC13DF0B08007D30FF
:1006C000DF00D60308003E1CDD123E18DD16BE1CFE
:1006D0005D12BE185D163E1DDD10DC18712B3E1933
:1006E000DD14BE1D5D10DC18772BBE195D14DC18FF
:1006F0005D10DC18DD10DE0B08000A30DE00521C35
:100700008512D21C0512DC18892B521D8510D21DB2
:1007100005103D18902BBD18902B0F30D20008000B
:10072000922308004D08D500ED23CD004E08D500DA
:10073000ED23CE004F08D5004D1CED23CF0050080F
:10074000D500CD1CED23D000C108031952140319A4
:10075000B52BC90BB52BCD1BC1034D08C900CD1856
:100760005214CD1E5210CD1D5210C2080319D214BE
:100770000319C62BCA0BC62BCE1BC2034E08CA00D8
:10078000CE1AD2144E1DD2104E1FD210BD18EC2B13
:10079000BD19EC2BC308031952150319DB2BCB0B26
:1007A000DB2BCF1BC3034F08CB004F1A52154F1F33
:1007B0005211CF1D5211C4080319D2150319EC2B85
:1007C000CC0BEC2BD01BC4035008CC00501AD21514
:1007D000D01FD211D01DD2110800C001D5080319B5
:1007E000D50355184014D51A40144008C001551CB3
:0E07F0004014D51E4014C005C00C550C080066
:084000000700000006000200A9
:02400E00CC01E3
:10420000010003000300030003000300020002009A
:104210000200020000000000FF00FF00FF00FF009E
:10422000000000000000000000000000000000008E
:1042300000000000C000C000FF00FF00FF00FF0002
:104240000000510005001500150055005100050043
:104250001500550051000500FF00FF00FF00FF00A2
:104260000000FF00FF00FF00FF00FF00FF00FF0055
:10427000FF00FF00FF00FF00FF00FF00FF00FF0046
:1042800002000F00FF00FF00FF00FF00FF00FF0023
:10429000FF00FF00FF00FF00FF00FF00FF00FF0026
:1042A000FF00FF00FF00FF00FF00FF00FF00FF0016
:1042B000FF00FF00FF00FF00FF00FF00FF00FF0006
:1042C000FF00FF00FF00FF00FF00FF00FF00FF00F6
:1042D000FF00FF00FF00FF00FF00FF00FF00FF00E6
:1042E000FF00FF00FF00FF00FF00FF00FF00FF00D6
:1042F000FF00FF00FF00FF00FF00FF00FF00AA001B
:00000001FF
